:0300000002118B5F
:03000B000200A54B
:03002B000202DEF0
:03005B000204BAE2
:03007300020489FB
:1000800002030406080C10182030406080040608A3
:100090000C10182030406080A0C00D0D0403060D28
:1000A0000503030202306306C26385768A32C2AF5B
:1000B000C0D0C0E020620C20680241BD3066024121
:1000C0007DE473C3E525334009758A00D263F57674
:1000D00001D4F58AC262E525F47002214420680249
:1000E000212B207213758B00758D00D0E0D0D0C20B
:1000F00093C297C294D2AF32C293C297C29474068D
:10010000D5E0FDE53C1420E21520E10D207D02D272
:1001100096307D02D29202013ED29502013E207DB0
:1001200002D292307D02D29602013E758B00758D0F
:1001300000D0E0D0D0C293C297C294D2AF32758BB8
:1001400000758D00D0E0D0D0D2AF3241BDE5256042
:100150000A207D02D293307D02D297C29441BDE540
:10016000256002D294207D02C297307D02C2934165
:10017000BDE525600A207D02D297307D02D2932012
:100180007D02C293307D02C29741BD207D02C292A2
:10019000307D02C296207D02C296307D02C29274EA
:1001A00006D5E0FDE525600A207D02D293307D0270
:1001B000D297C29441BD207D02C292307D02C29688
:1001C000C2957406D5E0FDE525600A207D02D29334
:1001D000307D02D297C29441BDC295207D02C29269
:1001E000307D02C2967406D5E0FDE5256002D2940A
:1001F000207D02C297307D02C29341BDC295207D11
:1002000002C296307D02C2927406D5E0FDE52560FB
:1002100002D294207D02C297307D02C29341BD205C
:100220007D02C296307D02C292C2957406D5E0FD71
:10023000E525600A207D02D297307D02D293207D91
:1002400002C293307D02C29741BD207D02C296302A
:100250007D02C292207D02C292307D02C296740657
:10026000D5E0FDE525600A207D02D297307D02D2DF
:1002700093207D02C293307D02C29741BD30723D12
:10028000E53C20E21A20E129207D02C292307D0265
:10029000C296207D02C296307D02C2920202BD202B
:1002A000E1E6207D02C292307D02C296C295020232
:1002B000BDC295207D02C296307D02C292E525F432
:1002C000C3334009758A00D263F57641CFF58A754C
:1002D0008B00758D00D262D0E0D0D0D2AF32C2AFE9
:1002E000C2AD53E6EFC0D0C0E0D2D3D2AFE5776065
:1002F00009E5746005757400618D757401C2CEE501
:100300002960072074461529614C78007900E58042
:10031000307E01F430E50278FF53DACF207E0343CC
:10032000DA20307E0343DA10C2D8C271E580307E15
:1003300001F430E50279FFC3E89970CE30610375AE
:1003400029402074037529408859D270E52A600439
:10035000152A615C20740543DA01C2D8207002615D
:1003600084A859206102C270207402616D88223015
:10037000690AC3E522955E4003855E227882B60451
:1003800003852224C3E52594404002D26420CF0C8B
:10039000D0E0D0D0C2D343E610D2AD32E5776009C9
:1003A000E5756005757500817D757501C2CF7802B0
:1003B000E52960053074021529C3E559940140050B
:1003C000755C0061D6755D00756400E55C2401F51F
:1003D0005C5003755CFF7982B7020EE547601EC36F
:1003E000E522943240178546227982B7030FE5470C
:1003F000600BC3E52294324004798E8722C3E52343
:100400009522600840041523810C0523D8C8056493
:10041000E56470021564D565647565017805C3E50A
:100420006495664058C3E564956750087801756522
:1004300003020440C3E564956850057801756501C1
:10044000C3E55F9524401F7982B704028172E547B6
:10045000701485245FE56404600385666475650136
:1004600075233C02047DE55F285005755FFF8172AE
:0F047000F55FE55F047006755DFF7564FFD0E012
:10047F00D0D0C2D343E610D2AD32C0D0C0E0C2AFAD
:10048F0053917F53E67FC260C3E55033F550E5517A
:10049F0033F551759100C3E49550F594E49551F5FA
:1004AF0095759104D0E0D0D0D2AF32C2AF53E6EF02
:1004BF00C2ADC0D0C0E0C0F0D2D3D2AFA8FBA9FC70
:1004CF00E5776007C3E913F9E813F8C2D830710272
:1004DF00A12C53DACF207E0343DA10307E0343DAA8
:1004EF0020D271E580307E01F420E502A103882639
:1004FF008927E10353DACF207E0343DA20307E03CE
:10050F0043DA10C2D8C271307402C1EF7800E580AF
:10051F00307E01F430E502C1EF8859C1D653DACFEE
:10052F00207E0343DA20307E0343DA10C27120614C
:10053F0002A1FC53DACF207E0343DA10307E03434F
:10054F00DA20C2D8D27188548955C3E89552F8E998
:10055F009553F9E4FB7E027A00C3E8948CE994008A
:10056F005005755800A1ECC3E894C8E994005008F1
:10057F00E4D2E4FB7A0AA1C9C3E89468E994015074
:10058F0008E4D2E3FB7A0FA1C9C3E894D0E994023F
:10059F005008E4D2E2FB7A1EA1C9C3E894A0E99403
:1005AF00055008E4D2E1FB7A3CA1C9C3E89498E96D
:1005BF0094085008E4D2E0FB7A787E00C3E89556A1
:1005CF00FCE99557FD30E708ECF42401FCEDF4FD50
:1005DF00755800C3EC9AED9E5003755801885689E3
:1005EF0057A854A955885289537802C1D6C3E895A4
:1005FF0026F8E99527F9307C02C1BA307B02C1BADF
:10060F00307A02C1B3207502C11FE9FDE8FCC13E7B
:10061F00E9C313F9E813F8307902C1B3E9C313F949
:10062F00E813F8307802C1B3E9C313FDE813FC20D7
:10063F006126C3EC941CED94024002C155ED701875
:10064F00C3EC94C850120528C3E528940A5002C180
:10065F00EF755900D270C1EFE528600215287400BC
:10066F00207F037896E624FAFEE43400FFC3EC9E65
:10067F00FCED9FFD500678007900C1BAC3EC94FFE2
:10068F00ED9400400678FF7900C1BAEC856FF0A4B5
:10069F00C5F0A2F733F8790040030206D678FF7948
:1006AF00000206D6E9C313F9E813F8307C0EE960AF
:1006BF000278FFC3E81338F8E43400F9C3E894FF75
:1006CF00E99400400278FF8859D270206102C1EF8F
:1006DF00741FF4552F4BF52FC274E42B7002D27494
:1006EF0075294030740375290A306102E1032074C3
:1006FF000353DAFE752A20307403752A0AD0F0D01E
:10070F00E0D0D0C2D3D2AD43E61032790102073820
:10071F007903020738790A020738791E02073879F8
:10072F006402073879C80207387817E4D5E0FDD896
:10073F00FAD9F6227A147B7802075F7A107B8C0243
:10074F00075F7A0D7BB402075F7A0B7BC802075FE6
:10075F00AC257525017902B27DE4C295D5E0FDE5A2
:10076F00256002D294D5E0FDC294D5E0FDD295D597
:10077F00E0FDE525600A207D02D293307D02D297FD
:10078F00E570D5E0FD207D02C293307D02C29774E3
:10079F0096D5E0FDD9C1EAF8D5E0FDD8FBDBB1C2B3
:1007AF00958C2522C37C007D0075F00005F0EA339F
:1007BF00FAEB33FB50F6EB13FBEA13FAC3E9FFE84E
:1007CF00FEE89AF8E99BF95004EFF9EEF8B3EC3331
:1007DF00FCED33FDD5F0DFEDF9ECF822E889F08A76
:1007EF0020D2D4F8A9F07B0030F70B7BFFF4240163
:1007FF00F8E9F43400F9E88520F0A4ADF0F8E985C4
:10080F0020F0A4AFF0FEED2EF974003FFA7C04C384
:10081F00EA13FAE913F9E813F8DCF48BF030F70A6E
:10082F00E8F42401F8E9F43400F9E889F0C2D4F8C7
:10083F00A9F0227882B604030208E4C3E55994199B
:10084F00401FE52D54067019E547703878057994E7
:10085F00E7146007780A1460027812C3E53B9840EA
:0E086F0020E547600985615F7564FF756501CE
:10087D00852224E4F53EF53FF540F541F542F54777
:10088D000208E47547017994E7147013E523F433F6
:10089D0033F913F8E9540104F9E854FE0208D8E7D6
:1008AD0014147014E523F4333333F913F8E95403B6
:1008BD0004F9E854FC0208E0E523F433333333F94B
:1008CD0013F8E954070404F9E854F8C39440F8E91F
:1008DD009400F9883E893F22E547603BC3E53B1311
:1008ED00F9E53A13F8C3E53E98F8E53F99F9500C50
:1008FD00C3E89480E994FF4016020920C3E8947F71
:10090D00E994005003020920787F790002092078CC
:10091D008079FF8843894422E5476058E5432540A7
:10092D00F8E5443541F9854420E4300701F43542BA
:10093D00FA30E709C3EA94F04015020962C3EA945C
:10094D000F500302096278FF79FF7A0F020962786E
:10095D000079007AF0C3E524955E5006E524600920
:10096D00217BE54420E70D217BE54430E7068840F7
:10097D0089418A4222E54770030209E678A1E6FA29
:10098D00C3E54333F8E54433F91207EBE930E70BE0
:10099D00C3E89480E994FF401321BDC3E8947FE937
:1009AD009400500221BD787F790021BD788079FFB8
:1009BD00E820E715C3E52398F84009C3E894014002
:1009CD00030209E478010209E4E8F424012523F87F
:1009DD0040030209E478FF884522E5477003020AC7
:1009ED004978A2E6FAA841A9421207EBE930E70CD3
:1009FD00C3E89401E994FF4016020A20C3E894FF6E
:100A0D00E994005003020A2078FF7900020A207849
:100A1D000179FFE920E715C3E54598F84009C3E8DA
:100A2D0094014003020A477800020A47E8F42401C2
:100A3D002545F84003020A4778FF88242278FFC233
:100A4D0064E52D5406702FD264C3E53B940A40092A
:100A5D00C3E52594405002C264E53B601974FF85DF
:100A6D003BF0848537F0A4F8C5F0600278FFC3E849
:100A7D0095615002A8618860227883E6F520120FF7
:100A8D00A975E89012071A75E890E5E820ECFBA827
:100A9D00BDA9BE121029756B01756C00C3740013CE
:100AAD00FD740113FC74012CFC74003DFDECFAED9A
:100ABD00FBC3E89AE99B4014E56B2401F56BE56CEB
:100ACD003400F56CEA2CFAEB3DFB80E5AE6BAF6CB8
:100ADD00C3E56C13F9E56B13F8C3E913F9E813F8E3
:100AED00E56B28F569E56C39F56A7A03C3E913F905
:100AFD00E813F8DAF7AA201A7009756B00756C0007
:100B0D00020B201AEA6008EE28FEEF39FFDAF88EA4
:100B1D006B8F6C2275E890227883E6FFE5E820EC78
:100B2D00F7A8BDA9BE056DC3E56D94084052756D5E
:100B3D0000E9FA79A0E76044EA7007E56E601B02F0
:100B4D000B5BC3E8956E6010E56E5006600C1402E9
:100B5D000B670460F9020B67E56EF56EC394724086
:100B6D001B755EC0C394044013755E80C39404402E
:100B7D000B755E40C394044003755E0075BB09227E
:100B8D00EFC39401601BC3E894FFE994035012C3B3
:100B9D00E8956BE9956C5009E55E600C155E020BEE
:100BAD00B5E55EF46002055EA85EC3E524985002CB
:100BBD00A824C3E8955F400AA85FE55FF46003854C
:100BCD005F5E8825E56DB4070375BB10227432791D
:100BDD00A387F0A4C5F0A2F733F8C3E8955E4002F1
:100BED00A85E882288248825886122753A00753B85
:100BFD007F2275C820A8CCA9CD75C824C3E913F9E7
:100C0D00E813F8AA38AB3988388939C3E89AF8E976
:100C1D009B547FF9AA3AAB3BAC3AAD3B7E047F02C5
:100C2D00C3EB940440021E1FC3EB940840021E1F29
:100C3D00C3ED13FDEC13FCDEF7C3EA9CFAEB9DFB51
:100C4D00EF6009C3E913F9E813F8DFF7EA28FAEBC7
:100C5D0039FB8A3A8B3B400122753AFF753BFF22E7
:0D0C6D00306002816D854C50854D51D26084
:100C7A0043E680227892E6FFC3E535948240010F6D
:100C8A00C3E53594A040010FC3EF940640027F05E7
:100C9A007E021E3072010EC3E53B940350060E0E0F
:100CAA003072010EC3E53B940250060E0E307201FB
:100CBA000EA93BA83A7A04C3E913F9E813F8DAF75C
:100CCA00C3E89EF8E99400F94009C3E89402E9945C
:100CDA000050047802E4F9E9FBE8FAC3E913FDE8F5
:100CEA0013FC884C894DC3EF94036037EF20E00D65
:100CFA00E82CF8E93DF9ECFAEDFB020D1AE828F8C0
:100D0A00E939F9C3E89402F8E99400F97A02E4FBB4
:100D1A00C3EF9403400D8A4E8B4F884889498C4A09
:100D2A008D4B22884E894F8A488B498C4A8D4B229B
:100D3A00306002A13AD26043E680E52D5406602E67
:100D4A00A83AA93BE53494085006E820E002A94DE8
:100D5A00C3E833F8E933F9759100C3E498F594E4EC
:100D6A0099F595759104D26053917F43E68022D21A
:100D7A0065753D00752000020D8CD265753D0075C4
:100D8A002040E52D54066002C265D2AF206005E519
:100D9A003D60012278017A02C3E53B94054002785E
:100DAA0002C3E53B940A40027803C3E53B940F4033
:100DBA00027A03306904781E7A01206007E53D60F3
:100DCA0003D2AF22D2AF0000C2AFC3E53BFB940F00
:100DDA0040027B0FEB043073012320620123F930B8
:100DEA0069027982E58D13E58B13C39940CC053DE1
:100DFA00EAFBE59BF45440B52004DBF6C1332065D9
:100E0A0002A18CC265759100AE3AAF3BC3EE33FEC8
:100E1A00EF33FFC3E49EF594E49FF595759104D2F0
:100E2A006053917F43E680A18C306502A18CD88AF9
:100E3A00D2AF2230690B0534206016753400020ED9
:100E4A005B20600D20650A206B071581158102164B
:100E5A005922A84EA94FC3E833F8E933F97591002E
:100E6A0053917FC3E498F594E499F59575910485B7
:100E7A004850854951D26043E680227800306405A3
:100E8A003065027801E53575F007A4F9E5F028F533
:100E9A00F0E9A2F013A2F113A2F213F535C3947884
:100EAA005003753578C3E53595364008D266C29346
:100EBA00C297C294306002C1BE854A50854B51D256
:100ECA006043E68022C2AFC292C296C29530720BCC
:100EDA0090021F7406D5E0FD020EE5207D02D29233
:100EEA00307D02D296759F80753C02021024C2AFF3
:100EFA00207D02C297307D02C2933072179001FCA6
:100F0A00C295207D02C296307D02C2927406D5E057
:100F1A00FD020F2190015F306206E5256002D2943E
:100F2A00207D03759F89307D03759F81753C03027F
:100F3A001024C2AFC292C296C29530720B9001D9E8
:100F4A007406D5E0FD020F52207D02D296307D0252
:100F5A00D292207D03759F81307D03759F89753CF0
:100F6A0004021024C2AFC2943072179001B6207DD9
:100F7A0002C292307D02C296C2957406D5E0FD0285
:100F8A000F8F90014D30620EE525600A207D02D256
:100F9A0093307D02D297759F80753C05021024C25A
:100FAA00AFC292C296C29530720B90018B7406D56D
:100FBA00E0FD020FBFD295207D03759F89307D0326
:100FCA00759F81753C06021024C2AF207D02C29330
:100FDA00307D02C29730721F90024A207D02C2926F
:100FEA00307D02C296207D02C296307D02C2927482
:100FFA0006D5E0FD02100490017130620EE525600D
:10100A000A207D02D297307D02D293207D03759FFC
:10101A0081307D03759F89753C01C266D2AF2290EB
:10102A00014BC293C297C294C292C296C295C2623F
:10103A00227880760708760708760108760408760B
:10104A00FF0876FF08760908760208760108760115
:10105A00788C76010876000876B40876FF0876FF61
:0F106A000876FF0876030876FF0876010876FF00
:101079000876250876D00876780876C808760408B0
:1010890076FF08760108760008767A08760A0876E7
:1010990001227887E6FFC272BF0302D2727888C242
:1010A9007DE630E102D27DC27E7889E630E102D266
:1010B9007EC3EF94026008758E01D2730210CD755C
:1010C9008E00C273227880E6149000809378A1F68E
:1010D9007881E6149000809378A2F6112922788607
:1010E900E61490008D9378A3F6112922789FE6F8EB
:1010F900700108C3E8941140027811E82828F566C0
:101109002566256628F56725662828F56822789CCE
:10111900E67536FF75370CB402067536A075370AC1
:10112900B4030675368275370522227896E6FA7871
:1011390097E6FB307F047A007BFFC3EB9AFCC394EC
:101149008250027C82756F00056FEC856FF0A4C335
:10115900E5F0948040F222D27F31341207297A00D7
:101169007B007C1012071FE5592AFA74003BFBDC4F
:10117900F37C04C3EB13FBEA13FADCF7FEC27F31FD
:101189003422E5EF20E6037520000520903FFFE5B6
:1011990020146006901FFF1460009304600375EF2C
:1011A90012C2D353D9BF7581C043FF8012071A7584
:1011B900EF0243B203E5B3240420E702F5B3112992
:1011C9007580FF75A40075F1F075D4DF759002750F
:1011D900A5FC75F2FD75D50275A61075A0FF75F30E
:1011E900F175E241113B12169B78988670C2AF12D5
:1011F900073312074312072912074A120729120750
:10120900511207291217BD12073312073312072E7D
:10121900C2AFE4F8F6D8FD78C879C8308507D9FB9C
:10122900D8F7021C00113B12169B119B11CE11E736
:1012390011F531173133313478988670112975B623
:101249008075A90075770075885075891275C8244D
:1012590075910475D84075A82275B80275E6907520
:101269009B80759D0075D10E75BCC075BB0975BA9B
:101279001175E88012071AD2AF120A8643DA01C241
:10128900D8C271120733753001D2617B037A0CE53C
:101299005870067A0CDB02411912072920700241A5
:1012A90019C270E559C3940240E3E52F541F855BC9
:1012B9005AF55BB55AD7DAD7C26153DACF207E0324
:1012C90043DA20307E0343DA10C2D8C271C2757581
:1012D900280012072E307409C3E528940A4002D267
:1012E9007512071F78023074027800C3E5599840D7
:1012F900F0C2AF120743120743120743D2AF1207D6
:101309003375460012071F788CE6C3940150030217
:1013190013E1E530C3940150030213E1207435C38E
:10132900E55994FF50030213E1C2AF120758D2AF37
:1013390012072EC3E559940150EFC2AF12074312A9
:101349000724120743D2AF12072EC3E55994FF4071
:10135900E90218427F05D27F313412072EC2AFC28B
:101369007F3134AE59C3E559947FD2AF4074120727
:101379001AC2AF120758D2AFDFDC3160C3EE940551
:101389007897F61207331216DC1217C57F0AD27F37
:10139900313412072EC2AFC27F3134AE59C3E55979
:1013A900947FD2AF50E612071AC2AF120743120751
:1013B90024120743D2AFDFD63160EE24057896F6C2
:1013C9001207331216DC1217F412072E3134C3E553
:1013D9005994FF40F4021842C3E5599546400385E4
:1013E900594612072E78017988E7B403027805C3B4
:1013F900E559984002610DC2AF12075812075812F9
:101409000758D2AF120733753000E4F531F53205CC
:1014190031E531F470390532789AE6781914601299
:10142900783214600D787D14600878FA14600375B9
:101439003200C3E53298401715327531B478998670
:1014490070C2AF120758D2AF7898867012072E1261
:101459000724E529700530740241197801207402C6
:0F1469007806C3E5599840A712072EE5297002AF
:101478004119C2AF1129E4F522F523F524F525D247
:10148800AF78858662F53EF53FF540F541F542F5C2
:101498006DF547F52CF52DF535120BF8756D0875BA
:1014A800BB1012071A120B21E5E820ECFBA8BDA916
:1014B800BEE97001F8886E120B25756D0875BB10B2
:1014C8007887E6FE7602119B7887EEF6C2AF755EE6
:1014D800FF120BDA85225E85225F852260D2AF7506
:1014E8002201752401752501855D6475650175B650
:1014F8009075A903757701D268D269753400120F07
:10150800A9120FD3120BF8120BFF120C7E02152230
:101518001129119B756D0075BB09120D84120E3DC2
:10152800120E5C120842120E85120ECF120BFF1219
:101538000C6D120C7E120D3A120D79120E3D120E20
:101548005C1208E5120A4A120E85120EF8120BFFF9
:10155800120C6D120C7E120D3A120D84120E3D12F1
:101568000E5C120925120E85120F3C120BFF120C8D
:101578006D120C7E120D3A120D79120E3D120E5C90
:10158800120982120E85120F6E120BFF120C6D12C9
:101598000C7E120D3A120D84120E3D120E5C1209C9
:1015A800E7120E85120FA9120BFF120C6D120C7E9A
:1015B800120D3A120D79120B21120E3D120E5C1209
:1015C8000B25120E85120FD3120BFF120C6D120C85
:1015D8007E120D3A30692F206B2C85615E85615F24
:1015E800855D6475650179327A0AC3E534994009E5
:1015F800C269D26A8A3302160EC3E55994014003C0
:10160800021522021659306A1B206B18E533147034
:1016180004C26AA118F533C3E559940140030215C1
:1016280022021659C3E55C9401400985615F855D16
:1016380064756501C3E55C94FA5016307404E529B5
:10164800600FC3E53B78F0306B027860985002A1D8
:1016580022C2AF11297887E6FE7602119B7887EEC1
:10166800F6E4F522F523F524F525F562C26875B68A
:101678008075A900757700D2AF12071A1129307446
:1016880006E52970024119788DE6C39401400241AC
:10169800EA8113901A0D782012171EE520B4A50CC4
:1016A800A312171EE520B45A030216BC113B1216EA
:1016B800DC0216DB901A0378807B0A12171EA30837
:1016C800DBF9901A0F788C7B1512171EA308DBF92B
:1016D800901A2422C2AF12175D121737901A00749D
:1016E8000D121723A37402121723A37413121723BE
:1016F800901A0378807B0A121722A308DBF9901A44
:101708000F788C7B15121722A308DBF912177012B9
:10171800174E901A2422E493F622E6438F01538F42
:10172800FD75EF0275B7A575B7F1F0538FFE22432B
:101738008F02438F0175EF0275B7A575B7F1901A3F
:101748000DF0538FFC22901A0D74A5F123901A0EF8
:10175800745AF123227A3079D07820901A40F11EF9
:10176800E520F709A3DAF7227A3079D0901A40E712
:10177800F12309A3DAF922AB71A872BB01027980BF
:10178800BB02027981BB03027982BB04027994BB54
:1017980005027983BB06027986BB07027992BB08EA
:1017A800027987BB0902799CBB0A027988BB0B02C4
:1017B8007989E8F7227C05120733DCFB22C2AF12D5
:1017C800074312074A120751120758120724120733
:1017D8004312074A120751120758120724120743E7
:1017E80012074A120751120758D2AF22C2AF120786
:1017F8005812075112074A120743120724120758B2
:1018080012075112074A12074312072412075812E7
:10181800075112074A120743D2AF22AE71AF72C204
:10182800AF120743120743120743120724DEF212CE
:101838000758120724DFF8D2AF221217C51217BDB6
:101848001217BD75710175720175730011237C053E
:10185800AD59120733C3ED955970F5C3E559940195
:0F186800400AC3E55994FF403702188512177FD5
:101877001216DC1217C5C2AF75EF121217BDDCD1F5
:101887000573C3E5739403500280C21217BD057236
:10189700E5711490009A93F808C3E5729850028096
:1018A700A91217BD1217BD0571C3E571940C50023B
:1018B700809512103B1216DCC2AF75EF121217BDDE
:101A00000D021307070104FFFF09020101A55A0196
:101A100000B4FFFFFF03FF01FF25D078C804FF01DA
:051A200000FF0A01FFB8
:101A40002358526F746F723430412320202020209D
:101A500023424C48454C492346333930232020202B
:101A60002020202020202020202020202020202076
:101C0000C2AFC2D353D9BF7581C043B20343FF8073
:101C1000752438752503B1BF75EF0275E24043F1B5
:101C20002053A4DFD285780379E67C1075220075F5
:101C30002300901DCC7B0675249875250130850204
:101C4000813D208508D8FBD9F9DCF781AD308508C6
:101C5000D8FBD9F9DCF781ADB17FE493A3C39A60D7
:101C6000028126DBDDB171600281267B08E493FAF4
:101C7000A3B152DBF87A30B152752200752300B15E
:101C800071EAFCEBFDC3ED94FE400EB1718A278B27
:101C900028ED30E0048A828B83B1717AC270D8C398
:101CA000ED94FE601050CEBD0022EC600675200061
:101CB0000200008100A827A9280809D804D90281B8
:101CC000C9B175EA89AAF281BB0D8199C3ED94036C
:101CD0005049EDA2E092007AC5C3E5829400E58305
:101CE000941C5093200010438F02438F0175B7A5B9
:101CF00075B7F1F030001FA827A9280809438F0104
:101D0000538FFDD804D902A11689AAE275B7A5752B
:101D1000B7F1F0A3A103538FFC81757AC1BD030C09
:101D2000E493A3FAB136DCF8B12E81758177AA224B
:101D3000AB23B152EBFAEA6222752608C3E52313FE
:101D4000F523E52213F52250066323A0632201D573
:101D500026EAB1BFB1BF75260AEAF4200102D28596
:101D6000300102C285B1BFC3134002C201D526EBC8
:101D700022B175EAFB208502A175308502A17A7532
:101D80002608AE24AF25C3EF13FFEE13FEB1C3B197
:101D9000BFC3EA133085024480FA30E703632201AF
:101DA000C3E52313F523E52213F52250066323A090
:101DB000632201D526D9E52265236523F52222AECB
:101DC00024AF250E0FDEFEDFFCD20122424C486517
:0A1DD0006C6934373132F3900601DC
:00000001FF
